:100000000C943B000C9450000C9450000C94500045
:100010000C9450000C9450000C9450000C94500020
:100020000C9450000C9450000C9450000C94500010
:100030000C9450000C9450000C9450000C94500000
:100040000C9450000C9450000C9450000C945000F0
:100050000C9450000C9450000C9450000C945000E0
:100060000C9450000C945000DA02DE02E202E50229
:10007000E902ED02DA0211241FBECFEFD8E0DEBFA5
:10008000CDBF11E0A0E0B1E0ECE8FBE002C00590DC
:100090000D92A430B107D9F70E9438030C94C4051F
:1000A0000C9400008C0181E087B9C0E0D0E0C0175B
:1000B000D1073CF440E060E085E50E9426012196EE
:1000C000F6CF2FEF86EB90E2215080409040E1F791
:1000D00000C00000C0E0D0E0C017D1073CF445E507
:1000E00060E080E00E9426012196F6CF2FEF86EB9C
:1000F00090E2215080409040E1F700C00000D5CF51
:100100002F923F924F925F926F927F928F929F9227
:10011000AF92BF92CF92DF92EF92FF920F931F9315
:10012000CF93DF93CDB7DEB72A970FB6F894DEBF33
:100130000FBECDBF78876F834A01190128013701AF
:100140002DB73EB73A8729879A01220F331F220F16
:10015000331F4DB75EB7421B530B0FB6F8945EBF0B
:100160000FBE4DBF2DB73EB72F5F3F4F3A83298358
:100170005C01C12CD12C8F819885C816D90641F11C
:100180004EE164E6C2010E9432036B837C838D835F
:100190009E834EE164E6C1010E943203E980FA8049
:1001A00084012B813C814D815E810E947701A401F5
:1001B000B50189819A810E940D03260C371C4618CF
:1001C00057083FEFC31AD30A4AE5A40EB11CD3CF98
:1001D00029853A850FB6F8943EBF0FBE2DBF2A96EB
:1001E0000FB6F894DEBF0FBECDBFDF91CF911F9148
:1001F0000F91FF90EF90DF90CF90BF90AF909F90C6
:100200008F907F906F905F904F903F902F900895C8
:1002100081E088B900C000C000C018B800C000C0AC
:1002200000C000C000C000C000C00000089581E010
:1002300088B900C000C000C000C000C000C000C03D
:1002400018B800C000C000C000C00895AF92BF92AF
:10025000CF92DF92EF92FF920F931F93CF93DF9392
:10026000C82EE42EC8E0D0E000E810E0A62EB12CA5
:10027000C8018A219B21892B19F00E94170102C015
:100280000E94080115950795219791F7C8E0D0E0E5
:1002900000E810E0D12CC8018C219D21892B19F098
:1002A0000E94170102C00E94080115950795219729
:1002B00091F7C8E0D0E000E810E0F12CC8018E21F1
:1002C0009F21892B19F00E94170102C00E9408018A
:1002D00015950795219791F7DF91CF911F910F9178
:1002E000FF90EF90DF90CF90BF90AF9008952F9246
:1002F0003F924F925F926F927F928F929F92AF92B6
:10030000BF92CF92DF92EF92FF920F931F93CF9302
:10031000DF93CDB7DEB72A970FB6F894DEBF0FBED6
:10032000CDBFD82EC92EF7010130110501F13B01D7
:100330002901461A570A842F90E0BC016D197109F2
:100340007E836D83852F90E09C012C1931093887BD
:100350002F8333961A861986E12CF12C80E090E0E9
:1003600020E030E0580141E0A41AB10805C06083E4
:100370007183828393833DC01C01240C351C4D8105
:100380005E814E0D5F1D5A8349834F815885698573
:100390007A85460F571F5C834B832017310749F13D
:1003A0004F0153E0851A9108B5010E949605660D2C
:1003B000771DD4016D937C934F01B1E08B1A9108A6
:1003C000C701B5010E9496056D0DD4016C93898516
:1003D0009A85B5010E9496056C0D60832F5F3F4F93
:1003E00034964B815C815A874987E980FA80C10144
:1003F000C3CF2A960FB6F894DEBF0FBECDBFDF91F4
:10040000CF911F910F91FF90EF90DF90CF90BF9011
:10041000AF909F908F907F906F905F904F903F90A4
:100420002F9008952F923F924F925F926F927F92FA
:100430008F929F92AF92BF92CF92DF92EF92FF92F4
:100440000F931F93CF93DF9300D000D0CDB7DEB7CB
:10045000FC01B2803380B11004C0232C3B823C826B
:10046000C2C0FC0100811181B8010836F1E01F070C
:1004700010F06856714080E090E00E949B042B01D0
:100480003C01632D70E080E090E00E949B0420E03E
:1004900030E048EC52E40E94FA036B017C016B2DC2
:1004A00070E080E090E00E949B0420E030E048ECA7
:1004B00052E40E94FA034B015C0120E030E040E787
:1004C00052E4C301B2010E94FA032B013C010E94D5
:1004D0006C046A8370E080E090E00E949D049B01C0
:1004E000AC01C301B2010E948D032B013C01A501A7
:1004F000940160E070E080E89FE30E948D039B011F
:10050000AC01C701B6010E94290520E030E040E0BF
:1005100053E40E9429050E946C04262EA301920137
:10052000C501B4010E9429059B01AC0160E070E0A7
:1005300080E89FE30E948D039B01AC01C701B601D7
:100540000E94290520E030E040E053E40E942905A4
:100550000E946C046983A301920160E070E080E86E
:100560009FE30E948D039B01AC01C501B4010E9471
:1005700029059B01AC0160E070E080E89FE30E94E8
:100580008D039B01AC01C701B6010E94290520E043
:1005900030E040E053E40E9429050E946C042A8167
:1005A000822F90E087309105E8F4FC01EC5CFF4F6E
:1005B0000C94AA052B826C83232C15C02B823C82C1
:1005C000298011C06B833C820EC03B8289818C8361
:1005D0000AC03B822C82262E06C0E981EB832C8246
:1005E000202E01C0212C622D7C818B810F900F90D9
:1005F0000F900F90DF91CF911F910F91FF90EF908F
:10060000DF90CF90BF90AF909F908F907F906F9032
:100610005F904F903F902F900895CF92DF92EF928E
:10062000FF920F931F93CF93DF936A01EB017C013D
:1006300000E010E00C151D0561F0C7010E941202D8
:100640006993799389930F5F1F4F84E0E80EF11C43
:10065000F1CFDF91CF911F910F91FF90EF90DF903D
:10066000CF900895282F862F622F792F942F0895E9
:10067000CF93DF931F92CDB7DEB78DB79EB7845B64
:100680009D420FB6F8949EBF0FBE8DBFEDB7FEB76B
:1006900031966F01EE24E394F12C02E612E02EE590
:1006A00031E04EE150E062E870E0CF010E9480004E
:1006B00081E087B991E000E010E02AE5922E909E5B
:1006C0005001919EB00C1124E12CF12CF701EA0DA0
:1006D000FB1DEC0DFD1D42816181808199830E948B
:1006E0002601F3E0EF0EF11C99818AE5E816F1048A
:1006F00069F7E7E8F3E13197F1F700C00000090F6F
:10070000111D97FD1A950238110511F49FEFD7CFEF
:1007100001151105A1F691E0D2CF5058BB27AA27A9
:100720000E94A5030C94EF040E94E10438F00E949B
:10073000E80420F039F49F3F19F426F40C94DE0409
:100740000EF4E095E7FB0C94D804E92F0E94000515
:1007500058F3BA17620773078407950720F079F4F6
:10076000A6F50C9422050EF4E0950B2EBA2FA02DC1
:100770000B01B90190010C01CA01A0011124FF274E
:10078000591B99F0593F50F4503E68F11A16F04049
:10079000A22F232F342F4427585FF3CF4695379548
:1007A0002795A795F0405395C9F77EF41F16BA0B0D
:1007B000620B730B840BBAF09150A1F0FF0FBB1FBB
:1007C000661F771F881FC2F70EC0BA0F621F731F04
:1007D000841F48F4879577956795B795F7959E3F61
:1007E00008F0B0CF9395880F08F09927EE0F9795F2
:1007F000879508950E940E040C94EF040E94E8046B
:1008000058F00E94E10440F029F45F3F29F00C9475
:10081000D80451110C9423050C94DE040E940005A9
:1008200068F39923B1F3552391F3951B550BBB271F
:10083000AA2762177307840738F09F5F5F4F220F64
:10084000331F441FAA1FA9F335D00E2E3AF0E0E85B
:1008500032D091505040E695001CCAF72BD0FE2FA5
:1008600029D0660F771F881FBB1F26173707480739
:10087000AB07B0E809F0BB0B802DBF01FF279358F1
:100880005F4F3AF09E3F510578F00C94D8040C94D9
:1008900023055F3FE4F3983ED4F3869577956795FB
:1008A000B795F7959F5FC9F7880F911D9695879526
:1008B00097F90895E1E0660F771F881FBB1F621745
:1008C00073078407BA0720F0621B730B840BBA0B03
:1008D000EE1F88F7E09508950E94080588F09F575D
:1008E00098F0B92F9927B751B0F0E1F0660F771F54
:1008F000881F991F1AF0BA95C9F714C0B13091F04A
:100900000E942205B1E008950C942205672F782FEC
:100910008827B85F39F0B93FCCF38695779567950E
:10092000B395D9F73EF490958095709561957F4F7A
:100930008F4F9F4F0895E89409C097FB3EF4909520
:100940008095709561957F4F8F4F9F4F9923A9F0A8
:10095000F92F96E9BB279395F69587957795679537
:10096000B795F111F8CFFAF4BB0F11F460FF1BC07B
:100970006F5F7F4F8F4F9F4F16C0882311F096E90E
:1009800011C0772321F09EE8872F762F05C06623BC
:1009900071F096E8862F70E060E02AF09A95660F75
:1009A000771F881FDAF7880F9695879597F908952E
:1009B00097F99F6780E870E060E008959FEF80EC12
:1009C000089500240A9416161706180609060895B5
:1009D00000240A9412161306140605060895092E1B
:1009E0000394000C11F4882352F0BB0F40F4BF2B8A
:1009F00011F460FF04C06F5F7F4F8F4F9F4F0895CA
:100A000057FD9058440F551F59F05F3F71F04795BF
:100A1000880F97FB991F61F09F3F79F087950895A4
:100A2000121613061406551FF2CF4695F1DF08C0C3
:100A3000161617061806991FF1CF869571056105E0
:100A400008940895E894BB2766277727CB0197F988
:100A500008950E943C050C94EF040E94E10438F0D4
:100A60000E94E80420F0952311F00C94D8040C9413
:100A7000DE0411240C9423050E94000570F3959F59
:100A8000C1F3950F50E0551F629FF001729FBB2785
:100A9000F00DB11D639FAA27F00DB11DAA1F649F21
:100AA0006627B00DA11D661F829F2227B00DA11DD4
:100AB000621F739FB00DA11D621F839FA00D611D5A
:100AC000221F749F3327A00D611D231F849F600D7B
:100AD000211D822F762F6A2F11249F5750409AF0A4
:100AE000F1F088234AF0EE0FFF1FBB1F661F771F30
:100AF000881F91505040A9F79E3F510580F00C94FB
:100B0000D8040C9423055F3FE4F3983ED4F3869514
:100B100077956795B795F795E7959F5FC1F7FE2B9A
:100B2000880F911D9695879597F9089597FB072E45
:100B300016F4009407D077FD09D00E94B00507FC99
:100B400005D03EF4909581959F4F089570956195DD
:100B50007F4F0895EE0FFF1F0590F491E02D09944B
:100B6000AA1BBB1B51E107C0AA1FBB1FA617B707D3
:100B700010F0A61BB70B881F991F5A95A9F78095EF
:0C0B80009095BC01CD010895F894FFCFC2
:040B8C0082001E00C5
:00000001FF
